:1000000010C02AC029C028C027C026C025C024C0CF
:1000100023C022C021C020C01FC01EC01DC01CC0E4
:1000200030C011241FBECFE5D1E0DEBFCDBF10E050
:10003000A0E6B0E0ECE4F4E002C005900D92A63634
:10004000B107D9F710E0A6E6B0E001C01D92AC36CA
:10005000B107E1F7A6D0F8C1D3CF20E030E040E00F
:1000600050E0A8E8B3E107C0FD013197F1F72F5F39
:100070003F4F4F4F5F4F2617370748075907A0F3E9
:1000800008951F920F920FB60F9211248F938091B3
:1000900066008FB910926600769A8F910F900FBE0E
:1000A0000F901F9018951FBC81E08EBD0895D798C2
:1000B000DF9A089589B3881F8827881F0895BA9802
:1000C00008954CB55DB5C29AB29BFECF2CB53DB537
:1000D000C298C901841B950B8F3F910519F010F050
:1000E0008FEF0895822F841B0895BA988EB584608F
:1000F0008EBD08952CB53DB5C298B299FECF8CB592
:100100009DB5C29A821B930B8F3F910511F008F0A9
:100110008FEF0895D19AD998D29ADA9A08954CB56A
:100120005DB5D198C99BFECF2CB53DB5D19AC9011B
:10013000841B950B8F3F910519F010F08FEF0895F8
:10014000822F841B0895D19AD99AD29ADA98089569
:100150004CB55DB5D198C999FECF2CB53DB5D19AB6
:10016000C901841B950B8F3F910519F010F08FEF9B
:100170000895822F841B0895D09AD89808958CB53D
:100180009DB5D098C89BFECF2CB53DB5D09A281B05
:10019000390B80E12030380710F02FEF3FE0C90124
:1001A0000895DF92EF92FF920F931F93CF93DF9307
:1001B000F894D39A8FEF88BB80E886BD16BC88E59B
:1001C0008DB9D59A8AB38F7A8ABB78941FBC81E0A7
:1001D0008EBDD798DF9AD09AD8980CB51DB5D09817
:1001E000C89BFECFCCB5DDB5D09A2CB53DB5D09827
:1001F000C89BFECF8CB59DB5D09AACB5BDB5D09897
:10020000C89BFECF6CB57DB5D09AECB5FDB5D09846
:10021000C89BFECF4CB55DB5D09A7C01E21AF30ABB
:10022000970180E12030380710F02FEF3FE0CE013A
:10023000801B910B10E18030910710F08FEF9FE051
:10024000280F391FCB018A1B9B0B60E1803096077A
:1002500010F08FEF9FE0280F391FCA018E1B9F0BF4
:1002600010E18030910710F08FEF9FE0820F931F15
:1002700020E18030920710F08FEF9FE065E170E0A1
:10028000D1D07C0180E3D82E8CB59DB51092690049
:1002900011C0E0916900F0E0E05AFF4F8081809347
:1002A0006600809166008823E1F7809169008F5F86
:1002B00080936900E0916900F0E0E05AFF4F80818F
:1002C000882339F710926600809166008823E1F751
:1002D0006CB57DB5D098C89BFECF2CB53DB5D09AF6
:1002E0000CB51DB5D098C89BFECFACB5BDB5D09AA6
:1002F000CCB5DDB5D098C89BFECFECB5FDB5D09A96
:100300004CB55DB5D098C89BFECF8CB59DB5D09A45
:10031000261B370B60E12030360710F02FEF3FE04F
:10032000841B950B40E18030940710F08FEF9FE025
:10033000280F391FCD01801B910B60E1803096079B
:1003400010F08FEF9FE0280F391FCF018C1B9D0B02
:1003500010E18030910710F08FEF9FE0280F391FD8
:1003600040E12030340710F02FEF3FE0D0926600DC
:10037000809166008823E1F7832F8F708A3010F414
:10038000805D01C0895C809366008091660088234F
:10039000E1F7922F822F82958F708A3010F4805D62
:1003A00001C0895C80936600809166008823E1F734
:1003B000892F8F708A3010F4805D01C0895C809332
:1003C0006600809166008823E1F71092690011C0F1
:1003D000E0916900F0E0EC59FF4F80818093660066
:1003E000809166008823E1F7809169008F5F809398
:1003F0006900E0916900F0E0EC59FF4F80818823AB
:1004000039F710926600809166008823E1F7C901F0
:1004100064E170E007D0E816F90610F4DB9A34CFF7
:10042000DB9832CF5527002480FF02C0060E571FED
:10043000660F771F6115710521F0969587950097D6
:0C04400099F7952F802D0895F894FFCFB8
:06044C0054333A000A00DF
:00000001FF
